


ARM Macro Assembler    Page 1 


    1 00000000         ;/******************************************************
                       ***********************
    2 00000000         ; * @file:    startup_MPS_CM3.s
    3 00000000         ; * @purpose: CMSIS Cortex-M3 Core Device Startup File 
    4 00000000         ; *           for the ARM 'Microcontroller Prototyping S
                       ystem' 
    5 00000000         ; * @version: V1.01
    6 00000000         ; * @date:    19. Aug. 2009
    7 00000000         ; *------- <<< Use Configuration Wizard in Context Menu 
                       >>> ------------------
    8 00000000         ; *
    9 00000000         ; * Copyright (C) 2008-2009 ARM Limited. All rights rese
                       rved.
   10 00000000         ; * ARM Limited (ARM) is supplying this software for use
                        with Cortex-M3 
   11 00000000         ; * processor based microcontrollers.  This file can be 
                       freely distributed 
   12 00000000         ; * within development tools that are supporting such AR
                       M based processors. 
   13 00000000         ; *
   14 00000000         ; * THIS SOFTWARE IS PROVIDED "AS IS".  NO WARRANTIES, W
                       HETHER EXPRESS, IMPLIED
   15 00000000         ; * OR STATUTORY, INCLUDING, BUT NOT LIMITED TO, IMPLIED
                        WARRANTIES OF
   16 00000000         ; * MERCHANTABILITY AND FITNESS FOR A PARTICULAR PURPOSE
                        APPLY TO THIS SOFTWARE.
   17 00000000         ; * ARM SHALL NOT, IN ANY CIRCUMSTANCES, BE LIABLE FOR S
                       PECIAL, INCIDENTAL, OR
   18 00000000         ; * CONSEQUENTIAL DAMAGES, FOR ANY REASON WHATSOEVER.
   19 00000000         ; *
   20 00000000         ; ******************************************************
                       ***********************/
   21 00000000         
   22 00000000         
   23 00000000         ; <h> Stack Configuration
   24 00000000         ;   <o> Stack Size (in Bytes) <0x0-0xFFFFFFFF:8>
   25 00000000         ; </h>
   26 00000000         
   27 00000000 00000200 
                       Stack_Size
                               EQU              0x00000200
   28 00000000         
   29 00000000                 AREA             STACK, NOINIT, READWRITE, ALIGN
=3
   30 00000000         Stack_Mem
                               SPACE            Stack_Size
   31 00000200         __initial_sp
   32 00000200         
   33 00000200         
   34 00000200         ; <h> Heap Configuration
   35 00000200         ;   <o>  Heap Size (in Bytes) <0x0-0xFFFFFFFF:8>
   36 00000200         ; </h>
   37 00000200         
   38 00000200 00000000 
                       Heap_Size
                               EQU              0x00000000
   39 00000200         
   40 00000200                 AREA             HEAP, NOINIT, READWRITE, ALIGN=
3



ARM Macro Assembler    Page 2 


   41 00000000         __heap_base
   42 00000000         Heap_Mem
                               SPACE            Heap_Size
   43 00000000         __heap_limit
   44 00000000         
   45 00000000         
   46 00000000                 PRESERVE8
   47 00000000                 THUMB
   48 00000000         
   49 00000000         ; FreeRTOS specific handlers.
   50 00000000                 EXTERN           vPortSVCHandler
   51 00000000                 EXTERN           xPortPendSVHandler
   52 00000000                 EXTERN           xPortSysTickHandler
   53 00000000         
   54 00000000         ; Vector Table Mapped to Address 0 at Reset
   55 00000000         
   56 00000000                 AREA             RESET, DATA, READONLY
   57 00000000                 EXPORT           __Vectors
   58 00000000         
   59 00000000 00000000 
                       __Vectors
                               DCD              __initial_sp ; Top of Stack
   60 00000004 00000000        DCD              Reset_Handler ; Reset Handler
   61 00000008 00000000        DCD              NMI_Handler ; NMI Handler
   62 0000000C 00000000        DCD              HardFault_Handler ; Hard Fault 
                                                            Handler
   63 00000010 00000000        DCD              MemManage_Handler 
                                                            ; MPU Fault Handler
                                                            
   64 00000014 00000000        DCD              BusFault_Handler 
                                                            ; Bus Fault Handler
                                                            
   65 00000018 00000000        DCD              UsageFault_Handler ; Usage Faul
                                                            t Handler
   66 0000001C 00000000        DCD              0           ; Reserved
   67 00000020 00000000        DCD              0           ; Reserved
   68 00000024 00000000        DCD              0           ; Reserved
   69 00000028 00000000        DCD              0           ; Reserved
   70 0000002C 00000000        DCD              vPortSVCHandler 
                                                            ; SVCall Handler
   71 00000030 00000000        DCD              DebugMon_Handler ; Debug Monito
                                                            r Handler
   72 00000034 00000000        DCD              0           ; Reserved
   73 00000038 00000000        DCD              xPortPendSVHandler 
                                                            ; PendSV Handler
   74 0000003C 00000000        DCD              xPortSysTickHandler 
                                                            ; SysTick Handler
   75 00000040         
   76 00000040         ; External Interrupts
   77 00000040 00000000        DCD              WDT_IRQHandler ; 0:  Watchdog T
                                                            imer
   78 00000044 00000000        DCD              RTC_IRQHandler ; 1:  Real Time 
                                                            Clock
   79 00000048 00000000        DCD              TIM0_IRQHandler ; 2:  Timer0 / 
                                                            Timer1
   80 0000004C 00000000        DCD              TIM2_IRQHandler ; 3:  Timer2 / 
                                                            Timer3
   81 00000050 00000000        DCD              MCIA_IRQHandler ; 4:  MCIa
   82 00000054 00000000        DCD              MCIB_IRQHandler ; 5:  MCIb



ARM Macro Assembler    Page 3 


   83 00000058 00000000        DCD              UART0_IRQHandler ; 6:  UART0 - 
                                                            DUT FPGA
   84 0000005C 00000000        DCD              UART1_IRQHandler ; 7:  UART1 - 
                                                            DUT FPGA
   85 00000060 00000000        DCD              UART2_IRQHandler ; 8:  UART2 - 
                                                            DUT FPGA
   86 00000064 00000000        DCD              UART4_IRQHandler ; 9:  UART4 - 
                                                            not connected
   87 00000068 00000000        DCD              AACI_IRQHandler 
                                                            ; 10: AACI / AC97
   88 0000006C 00000000        DCD              CLCD_IRQHandler ; 11: CLCD Comb
                                                            ined Interrupt
   89 00000070 00000000        DCD              ENET_IRQHandler ; 12: Ethernet
   90 00000074 00000000        DCD              USBDC_IRQHandler 
                                                            ; 13: USB Device
   91 00000078 00000000        DCD              USBHC_IRQHandler ; 14: USB Host
                                                             Controller
   92 0000007C 00000000        DCD              CHLCD_IRQHandler 
                                                            ; 15: Character LCD
                                                            
   93 00000080 00000000        DCD              FLEXRAY_IRQHandler 
                                                            ; 16: Flexray
   94 00000084 00000000        DCD              CAN_IRQHandler ; 17: CAN
   95 00000088 00000000        DCD              LIN_IRQHandler ; 18: LIN
   96 0000008C 00000000        DCD              I2C_IRQHandler 
                                                            ; 19: I2C ADC/DAC
   97 00000090 00000000        DCD              0           ; 20: Reserved
   98 00000094 00000000        DCD              0           ; 21: Reserved
   99 00000098 00000000        DCD              0           ; 22: Reserved
  100 0000009C 00000000        DCD              0           ; 23: Reserved
  101 000000A0 00000000        DCD              0           ; 24: Reserved
  102 000000A4 00000000        DCD              0           ; 25: Reserved
  103 000000A8 00000000        DCD              0           ; 26: Reserved
  104 000000AC 00000000        DCD              0           ; 27: Reserved
  105 000000B0 00000000        DCD              CPU_CLCD_IRQHandler ; 28: Reser
                                                            ved - CPU FPGA CLCD
                                                            
  106 000000B4 00000000        DCD              0           ; 29: Reserved - CP
                                                            U FPGA
  107 000000B8 00000000        DCD              UART3_IRQHandler ; 30: UART3   
                                                             - CPU FPGA
  108 000000BC 00000000        DCD              SPI_IRQHandler ; 31: SPI Touchs
                                                            creen - CPU FPGA
  109 000000C0         
  110 000000C0         
  111 000000C0                 AREA             |.text|, CODE, READONLY
  112 00000000         
  113 00000000         
  114 00000000         ; Reset Handler
  115 00000000         
  116 00000000         Reset_Handler
                               PROC
  117 00000000                 EXPORT           Reset_Handler             [WEAK
]
  118 00000000                 IMPORT           __main
  119 00000000 4805            LDR              R0, =__main
  120 00000002 4700            BX               R0
  121 00000004                 ENDP
  122 00000004         



ARM Macro Assembler    Page 4 


  123 00000004         
  124 00000004         ; Dummy Exception Handlers (infinite loops which can be 
                       modified)
  125 00000004         
  126 00000004         NMI_Handler
                               PROC
  127 00000004                 EXPORT           NMI_Handler               [WEAK
]
  128 00000004 E7FE            B                .
  129 00000006                 ENDP
  131 00000006         HardFault_Handler
                               PROC
  132 00000006                 EXPORT           HardFault_Handler         [WEAK
]
  133 00000006 E7FE            B                .
  134 00000008                 ENDP
  136 00000008         MemManage_Handler
                               PROC
  137 00000008                 EXPORT           MemManage_Handler         [WEAK
]
  138 00000008 E7FE            B                .
  139 0000000A                 ENDP
  141 0000000A         BusFault_Handler
                               PROC
  142 0000000A                 EXPORT           BusFault_Handler          [WEAK
]
  143 0000000A E7FE            B                .
  144 0000000C                 ENDP
  146 0000000C         UsageFault_Handler
                               PROC
  147 0000000C                 EXPORT           UsageFault_Handler        [WEAK
]
  148 0000000C E7FE            B                .
  149 0000000E                 ENDP
  150 0000000E         SVC_Handler
                               PROC
  151 0000000E                 EXPORT           SVC_Handler               [WEAK
]
  152 0000000E E7FE            B                .
  153 00000010                 ENDP
  155 00000010         DebugMon_Handler
                               PROC
  156 00000010                 EXPORT           DebugMon_Handler          [WEAK
]
  157 00000010 E7FE            B                .
  158 00000012                 ENDP
  159 00000012         PendSV_Handler
                               PROC
  160 00000012                 EXPORT           PendSV_Handler            [WEAK
]
  161 00000012 E7FE            B                .
  162 00000014                 ENDP
  163 00000014         SysTick_Handler
                               PROC
  164 00000014                 EXPORT           SysTick_Handler           [WEAK
]
  165 00000014 E7FE            B                .
  166 00000016                 ENDP
  167 00000016         



ARM Macro Assembler    Page 5 


  168 00000016         Default_Handler
                               PROC
  169 00000016         
  170 00000016                 EXPORT           WDT_IRQHandler            [WEAK
]
  171 00000016                 EXPORT           RTC_IRQHandler            [WEAK
]
  172 00000016                 EXPORT           TIM0_IRQHandler           [WEAK
]
  173 00000016                 EXPORT           TIM2_IRQHandler           [WEAK
]
  174 00000016                 EXPORT           MCIA_IRQHandler           [WEAK
]
  175 00000016                 EXPORT           MCIB_IRQHandler           [WEAK
]
  176 00000016                 EXPORT           UART0_IRQHandler          [WEAK
]
  177 00000016                 EXPORT           UART1_IRQHandler          [WEAK
]
  178 00000016                 EXPORT           UART2_IRQHandler          [WEAK
]
  179 00000016                 EXPORT           UART3_IRQHandler          [WEAK
]
  180 00000016                 EXPORT           UART4_IRQHandler          [WEAK
]
  181 00000016                 EXPORT           AACI_IRQHandler           [WEAK
]
  182 00000016                 EXPORT           CLCD_IRQHandler           [WEAK
]
  183 00000016                 EXPORT           ENET_IRQHandler           [WEAK
]
  184 00000016                 EXPORT           USBDC_IRQHandler          [WEAK
]
  185 00000016                 EXPORT           USBHC_IRQHandler          [WEAK
]
  186 00000016                 EXPORT           CHLCD_IRQHandler          [WEAK
]
  187 00000016                 EXPORT           FLEXRAY_IRQHandler        [WEAK
]
  188 00000016                 EXPORT           CAN_IRQHandler            [WEAK
]
  189 00000016                 EXPORT           LIN_IRQHandler            [WEAK
]
  190 00000016                 EXPORT           I2C_IRQHandler            [WEAK
]
  191 00000016                 EXPORT           CPU_CLCD_IRQHandler       [WEAK
]
  192 00000016                 EXPORT           SPI_IRQHandler            [WEAK
]
  193 00000016         
  194 00000016         WDT_IRQHandler
  195 00000016         RTC_IRQHandler
  196 00000016         TIM0_IRQHandler
  197 00000016         TIM2_IRQHandler
  198 00000016         MCIA_IRQHandler
  199 00000016         MCIB_IRQHandler
  200 00000016         UART0_IRQHandler
  201 00000016         UART1_IRQHandler
  202 00000016         UART2_IRQHandler



ARM Macro Assembler    Page 6 


  203 00000016         UART3_IRQHandler
  204 00000016         UART4_IRQHandler
  205 00000016         AACI_IRQHandler
  206 00000016         CLCD_IRQHandler
  207 00000016         ENET_IRQHandler
  208 00000016         USBDC_IRQHandler
  209 00000016         USBHC_IRQHandler
  210 00000016         CHLCD_IRQHandler
  211 00000016         FLEXRAY_IRQHandler
  212 00000016         CAN_IRQHandler
  213 00000016         LIN_IRQHandler
  214 00000016         I2C_IRQHandler
  215 00000016         CPU_CLCD_IRQHandler
  216 00000016         SPI_IRQHandler
  217 00000016 E7FE            B                .
  218 00000018         
  219 00000018                 ENDP
  220 00000018         
  221 00000018         
  222 00000018                 ALIGN
  223 00000018         
  224 00000018         
  225 00000018         ; User Initial Stack & Heap
  226 00000018         
  227 00000018                 IF               :DEF:__MICROLIB
  228 00000018         
  229 00000018                 EXPORT           __initial_sp
  230 00000018                 EXPORT           __heap_base
  231 00000018                 EXPORT           __heap_limit
  232 00000018         
  233 00000018                 ELSE
  247                          ENDIF
  248 00000018         
  249 00000018         
  250 00000018                 END
              00000000 
Command Line: --debug --xref --diag_suppress=9931 --cpu=Cortex-M3 --apcs=interw
ork --depend=.\keil_output\startup_mps_cm3.d -o.\keil_output\startup_mps_cm3.o 
-I.\RTE\_lab001 -IC:\Keil_v5\ARM\PACK\ARM\CMSIS\5.0.1\CMSIS\Include -IC:\Keil_v
5\ARM\PACK\Keil\LPC1700_DFP\2.3.0\Device\Include --predefine="__EVAL SETA 1" --
predefine="__MICROLIB SETA 1" --predefine="__UVISION_VERSION SETA 524" --predef
ine="_RTE_ SETA 1" --predefine="LPC175x_6x SETA 1" --list=.\keil_output\startup
_mps_cm3.lst startup_MPS_CM3.s



ARM Macro Assembler    Page 1 Alphabetic symbol ordering
Relocatable symbols

STACK 00000000

Symbol: STACK
   Definitions
      At line 29 in file startup_MPS_CM3.s
   Uses
      None
Comment: STACK unused
Stack_Mem 00000000

Symbol: Stack_Mem
   Definitions
      At line 30 in file startup_MPS_CM3.s
   Uses
      None
Comment: Stack_Mem unused
__initial_sp 00000200

Symbol: __initial_sp
   Definitions
      At line 31 in file startup_MPS_CM3.s
   Uses
      At line 59 in file startup_MPS_CM3.s
      At line 229 in file startup_MPS_CM3.s

3 symbols



ARM Macro Assembler    Page 1 Alphabetic symbol ordering
Relocatable symbols

HEAP 00000000

Symbol: HEAP
   Definitions
      At line 40 in file startup_MPS_CM3.s
   Uses
      None
Comment: HEAP unused
Heap_Mem 00000000

Symbol: Heap_Mem
   Definitions
      At line 42 in file startup_MPS_CM3.s
   Uses
      None
Comment: Heap_Mem unused
__heap_base 00000000

Symbol: __heap_base
   Definitions
      At line 41 in file startup_MPS_CM3.s
   Uses
      At line 230 in file startup_MPS_CM3.s
Comment: __heap_base used once
__heap_limit 00000000

Symbol: __heap_limit
   Definitions
      At line 43 in file startup_MPS_CM3.s
   Uses
      At line 231 in file startup_MPS_CM3.s
Comment: __heap_limit used once
4 symbols



ARM Macro Assembler    Page 1 Alphabetic symbol ordering
Relocatable symbols

RESET 00000000

Symbol: RESET
   Definitions
      At line 56 in file startup_MPS_CM3.s
   Uses
      None
Comment: RESET unused
__Vectors 00000000

Symbol: __Vectors
   Definitions
      At line 59 in file startup_MPS_CM3.s
   Uses
      At line 57 in file startup_MPS_CM3.s
Comment: __Vectors used once
2 symbols



ARM Macro Assembler    Page 1 Alphabetic symbol ordering
Relocatable symbols

.text 00000000

Symbol: .text
   Definitions
      At line 111 in file startup_MPS_CM3.s
   Uses
      None
Comment: .text unused
AACI_IRQHandler 00000016

Symbol: AACI_IRQHandler
   Definitions
      At line 205 in file startup_MPS_CM3.s
   Uses
      At line 87 in file startup_MPS_CM3.s
      At line 181 in file startup_MPS_CM3.s

BusFault_Handler 0000000A

Symbol: BusFault_Handler
   Definitions
      At line 141 in file startup_MPS_CM3.s
   Uses
      At line 64 in file startup_MPS_CM3.s
      At line 142 in file startup_MPS_CM3.s

CAN_IRQHandler 00000016

Symbol: CAN_IRQHandler
   Definitions
      At line 212 in file startup_MPS_CM3.s
   Uses
      At line 94 in file startup_MPS_CM3.s
      At line 188 in file startup_MPS_CM3.s

CHLCD_IRQHandler 00000016

Symbol: CHLCD_IRQHandler
   Definitions
      At line 210 in file startup_MPS_CM3.s
   Uses
      At line 92 in file startup_MPS_CM3.s
      At line 186 in file startup_MPS_CM3.s

CLCD_IRQHandler 00000016

Symbol: CLCD_IRQHandler
   Definitions
      At line 206 in file startup_MPS_CM3.s
   Uses
      At line 88 in file startup_MPS_CM3.s
      At line 182 in file startup_MPS_CM3.s

CPU_CLCD_IRQHandler 00000016

Symbol: CPU_CLCD_IRQHandler
   Definitions
      At line 215 in file startup_MPS_CM3.s
   Uses



ARM Macro Assembler    Page 2 Alphabetic symbol ordering
Relocatable symbols

      At line 105 in file startup_MPS_CM3.s
      At line 191 in file startup_MPS_CM3.s

DebugMon_Handler 00000010

Symbol: DebugMon_Handler
   Definitions
      At line 155 in file startup_MPS_CM3.s
   Uses
      At line 71 in file startup_MPS_CM3.s
      At line 156 in file startup_MPS_CM3.s

Default_Handler 00000016

Symbol: Default_Handler
   Definitions
      At line 168 in file startup_MPS_CM3.s
   Uses
      None
Comment: Default_Handler unused
ENET_IRQHandler 00000016

Symbol: ENET_IRQHandler
   Definitions
      At line 207 in file startup_MPS_CM3.s
   Uses
      At line 89 in file startup_MPS_CM3.s
      At line 183 in file startup_MPS_CM3.s

FLEXRAY_IRQHandler 00000016

Symbol: FLEXRAY_IRQHandler
   Definitions
      At line 211 in file startup_MPS_CM3.s
   Uses
      At line 93 in file startup_MPS_CM3.s
      At line 187 in file startup_MPS_CM3.s

HardFault_Handler 00000006

Symbol: HardFault_Handler
   Definitions
      At line 131 in file startup_MPS_CM3.s
   Uses
      At line 62 in file startup_MPS_CM3.s
      At line 132 in file startup_MPS_CM3.s

I2C_IRQHandler 00000016

Symbol: I2C_IRQHandler
   Definitions
      At line 214 in file startup_MPS_CM3.s
   Uses
      At line 96 in file startup_MPS_CM3.s
      At line 190 in file startup_MPS_CM3.s

LIN_IRQHandler 00000016

Symbol: LIN_IRQHandler



ARM Macro Assembler    Page 3 Alphabetic symbol ordering
Relocatable symbols

   Definitions
      At line 213 in file startup_MPS_CM3.s
   Uses
      At line 95 in file startup_MPS_CM3.s
      At line 189 in file startup_MPS_CM3.s

MCIA_IRQHandler 00000016

Symbol: MCIA_IRQHandler
   Definitions
      At line 198 in file startup_MPS_CM3.s
   Uses
      At line 81 in file startup_MPS_CM3.s
      At line 174 in file startup_MPS_CM3.s

MCIB_IRQHandler 00000016

Symbol: MCIB_IRQHandler
   Definitions
      At line 199 in file startup_MPS_CM3.s
   Uses
      At line 82 in file startup_MPS_CM3.s
      At line 175 in file startup_MPS_CM3.s

MemManage_Handler 00000008

Symbol: MemManage_Handler
   Definitions
      At line 136 in file startup_MPS_CM3.s
   Uses
      At line 63 in file startup_MPS_CM3.s
      At line 137 in file startup_MPS_CM3.s

NMI_Handler 00000004

Symbol: NMI_Handler
   Definitions
      At line 126 in file startup_MPS_CM3.s
   Uses
      At line 61 in file startup_MPS_CM3.s
      At line 127 in file startup_MPS_CM3.s

PendSV_Handler 00000012

Symbol: PendSV_Handler
   Definitions
      At line 159 in file startup_MPS_CM3.s
   Uses
      At line 160 in file startup_MPS_CM3.s
Comment: PendSV_Handler used once
RTC_IRQHandler 00000016

Symbol: RTC_IRQHandler
   Definitions
      At line 195 in file startup_MPS_CM3.s
   Uses
      At line 78 in file startup_MPS_CM3.s
      At line 171 in file startup_MPS_CM3.s




ARM Macro Assembler    Page 4 Alphabetic symbol ordering
Relocatable symbols

Reset_Handler 00000000

Symbol: Reset_Handler
   Definitions
      At line 116 in file startup_MPS_CM3.s
   Uses
      At line 60 in file startup_MPS_CM3.s
      At line 117 in file startup_MPS_CM3.s

SPI_IRQHandler 00000016

Symbol: SPI_IRQHandler
   Definitions
      At line 216 in file startup_MPS_CM3.s
   Uses
      At line 108 in file startup_MPS_CM3.s
      At line 192 in file startup_MPS_CM3.s

SVC_Handler 0000000E

Symbol: SVC_Handler
   Definitions
      At line 150 in file startup_MPS_CM3.s
   Uses
      At line 151 in file startup_MPS_CM3.s
Comment: SVC_Handler used once
SysTick_Handler 00000014

Symbol: SysTick_Handler
   Definitions
      At line 163 in file startup_MPS_CM3.s
   Uses
      At line 164 in file startup_MPS_CM3.s
Comment: SysTick_Handler used once
TIM0_IRQHandler 00000016

Symbol: TIM0_IRQHandler
   Definitions
      At line 196 in file startup_MPS_CM3.s
   Uses
      At line 79 in file startup_MPS_CM3.s
      At line 172 in file startup_MPS_CM3.s

TIM2_IRQHandler 00000016

Symbol: TIM2_IRQHandler
   Definitions
      At line 197 in file startup_MPS_CM3.s
   Uses
      At line 80 in file startup_MPS_CM3.s
      At line 173 in file startup_MPS_CM3.s

UART0_IRQHandler 00000016

Symbol: UART0_IRQHandler
   Definitions
      At line 200 in file startup_MPS_CM3.s
   Uses
      At line 83 in file startup_MPS_CM3.s



ARM Macro Assembler    Page 5 Alphabetic symbol ordering
Relocatable symbols

      At line 176 in file startup_MPS_CM3.s

UART1_IRQHandler 00000016

Symbol: UART1_IRQHandler
   Definitions
      At line 201 in file startup_MPS_CM3.s
   Uses
      At line 84 in file startup_MPS_CM3.s
      At line 177 in file startup_MPS_CM3.s

UART2_IRQHandler 00000016

Symbol: UART2_IRQHandler
   Definitions
      At line 202 in file startup_MPS_CM3.s
   Uses
      At line 85 in file startup_MPS_CM3.s
      At line 178 in file startup_MPS_CM3.s

UART3_IRQHandler 00000016

Symbol: UART3_IRQHandler
   Definitions
      At line 203 in file startup_MPS_CM3.s
   Uses
      At line 107 in file startup_MPS_CM3.s
      At line 179 in file startup_MPS_CM3.s

UART4_IRQHandler 00000016

Symbol: UART4_IRQHandler
   Definitions
      At line 204 in file startup_MPS_CM3.s
   Uses
      At line 86 in file startup_MPS_CM3.s
      At line 180 in file startup_MPS_CM3.s

USBDC_IRQHandler 00000016

Symbol: USBDC_IRQHandler
   Definitions
      At line 208 in file startup_MPS_CM3.s
   Uses
      At line 90 in file startup_MPS_CM3.s
      At line 184 in file startup_MPS_CM3.s

USBHC_IRQHandler 00000016

Symbol: USBHC_IRQHandler
   Definitions
      At line 209 in file startup_MPS_CM3.s
   Uses
      At line 91 in file startup_MPS_CM3.s
      At line 185 in file startup_MPS_CM3.s

UsageFault_Handler 0000000C

Symbol: UsageFault_Handler



ARM Macro Assembler    Page 6 Alphabetic symbol ordering
Relocatable symbols

   Definitions
      At line 146 in file startup_MPS_CM3.s
   Uses
      At line 65 in file startup_MPS_CM3.s
      At line 147 in file startup_MPS_CM3.s

WDT_IRQHandler 00000016

Symbol: WDT_IRQHandler
   Definitions
      At line 194 in file startup_MPS_CM3.s
   Uses
      At line 77 in file startup_MPS_CM3.s
      At line 170 in file startup_MPS_CM3.s

35 symbols



ARM Macro Assembler    Page 1 Alphabetic symbol ordering
Absolute symbols

Heap_Size 00000000

Symbol: Heap_Size
   Definitions
      At line 38 in file startup_MPS_CM3.s
   Uses
      At line 42 in file startup_MPS_CM3.s
Comment: Heap_Size used once
Stack_Size 00000200

Symbol: Stack_Size
   Definitions
      At line 27 in file startup_MPS_CM3.s
   Uses
      At line 30 in file startup_MPS_CM3.s
Comment: Stack_Size used once
2 symbols



ARM Macro Assembler    Page 1 Alphabetic symbol ordering
External symbols

__main 00000000

Symbol: __main
   Definitions
      At line 118 in file startup_MPS_CM3.s
   Uses
      At line 119 in file startup_MPS_CM3.s
Comment: __main used once
vPortSVCHandler 00000000

Symbol: vPortSVCHandler
   Definitions
      At line 50 in file startup_MPS_CM3.s
   Uses
      At line 70 in file startup_MPS_CM3.s
Comment: vPortSVCHandler used once
xPortPendSVHandler 00000000

Symbol: xPortPendSVHandler
   Definitions
      At line 51 in file startup_MPS_CM3.s
   Uses
      At line 73 in file startup_MPS_CM3.s
Comment: xPortPendSVHandler used once
xPortSysTickHandler 00000000

Symbol: xPortSysTickHandler
   Definitions
      At line 52 in file startup_MPS_CM3.s
   Uses
      At line 74 in file startup_MPS_CM3.s
Comment: xPortSysTickHandler used once
4 symbols
387 symbols in table
